:10000000830100308A003D28DB0003088301DC0007
:1000100083122A088100A90AAB0A1F30AB05003001
:100020008A002B08162086000B1137288207083417
:1000300009340A340C340D340E340E340F340F34BA
:100040000F340E340E340D340C340A3409340834B1
:1000500006340534033402340134013400340034EE
:10006000003401340134023403340534063483127D
:100070005C088300DB0E5B0E0900213084005130E8
:100080005320203084002130532083010730DA00D0
:10009000F830D90051308400593057208301462D63
:1000A00004068001840A0406031D50280034F00071
:1000B00062208000840A040870060319003458285E
:1000C0008312D900DA1B6B285A088A005908D90A0A
:1000D0000319DA0A820083135A1883175908D90AB8
:0600E00084000008080086
:100672008312EC232C3A8312031908003A2B8316B7
:100682009B001C148312CF0083161A0883120800E1
:10069200F0000030711870070310F00D0310F10C18
:1006A200F108031908004B2BF401F5010310F30CB8
:1006B200F20C031C632B7008F40771080318710A0B
:1006C200F5070310F00DF10D7208730403190034DD
:1006D200572B8511A01985158312CF000A30CE0041
:1006E2005130AE00861F792B5930AE07AE0B772BF7
:1006F200640083124F1C822B8515A01D862B851149
:10070200862B8511A01D862B851503148312CF0C11
:10071200CE0B712B0800CD01CE01CF01D000AE2B44
:100722000A30F200F3014E08F1004D08F0005523A3
:100732004F08500784000008F000F1017408F00728
:100742000318F10A7508F107D0307007CD00FF30A9
:10075200031800307107CE00CF0A033083124F0214
:10076200031C912B4E08F1004D08F00008004130A7
:100772006A2354306A2308306A230230DE2BEC23CA
:10078200CD0083169C18C32B83124D0883169B0041
:100792008312EC2383169A0003108B1B03148B1312
:1007A20083161C1555309D00AA309D009C141C1107
:1007B20003188B1783124D0840236A238312EC23FC
:1007C200CD00573A0319C02B83124D08523A031D2C
:1007D2000800EC23DD2BF32B6400061EF22B051020
:1007E200F42B05148312051AF82BA019ED2B051E04
:0E07F200FC2BA01DED2BCE012830AE00AE0B6F
:10080000FF2B0830CF0064008312861F092CAA300A
:100810000A2C5130AE00AE0B0B2C03108312CE0C01
:10082000A01D152C051A182C172C051E182CCE17D8
:10083000CF0B032C861F1E2CAA301F2C5130AE006C
:10084000AE0B202C8312A019051E272C2A2CA01DCC
:10085000051A2C2C0830A0064E080800CF01D00045
:1008600008304F0283120318080020115018201579
:100870000310A01C502CA70CA80C201D412C0130EB
:10088000422C0030F000031C472C0130482C003073
:10089000F00603194F2C8430A7060830A806031071
:1008A0008312D00CA01E5A2C640020302902031899
:1008B0005F2C542C64003A302902031C5A2CA901E5
:1008C000201D772CAC0A201E802C2C08053A031D15
:1008D000802CA01E712C6400203029020318762C75
:1008E0006B2C64003A302902031C712CA901A01A58
:1008F0007B2CCA307C2CE730AA002030A006AC014B
:10090000CF0A08304F0203180800352CCD01CD0A5C
:100910009C2C6400061A902CCD01CD0A0514912C54
:100920000510CE0120304E0203189B2CCE0A203039
:100930004E02031C962CCD0A8312CD08031D892C70
:100940000515A012831681158112C630831281000D
:100950008B17FF30A800A700A0101D304023CD004A
:100960008312CD080319B82C00302E24CD03B02CEF
:100970007E302E24A0142016AC01CD018312CD0AA6
:100980004D034023CE002E244E1CBE2C0330831278
:100990002E24F0302E2421302E24CD0108304D029B
:1009A0000318DA2C83124D08393E840000082E24E7
:1009B000CD0ACE2C1E30831240232E24CD010930C7
:1009C0004D020318EB2C83124D08413E84000008B1
:1009D0002E24CD0ADF2C1F30831240232E24CD017C
:1009E00003304D020318FC2C83124D08513E840045
:1009F00000082E24CD0AF02C2F3083122E24CD0196
:100A000003304D0203180C2D83124D08543E840010
:100A100000082E24CD0A002D2F3083122E244130C1
:100A20002E243D302E242608303E2E242508303E2C
:100A30002E242408303E2E242308303E2E24220863
:100A4000303E2E242108303E2E2420302E2420300B
:100A5000CD008312CD0A4D034023CE00CE08831271
:100A60000319352D4E082E24292DA010FF30A8067D
:100A7000A70628082E2427082E2420127E302E2494
:100A80007E302E2405118B138312080064008B0125
:100A90008B1607309F008316811310308500F030CD
:100AA00086008312051485140511602D4A08213A29
:100AB000031D602DB823602D4A08563A03195F2E96
:100AC00064008312EC23CA00243A031D562D8312BE
:100AD000EC23473A031D602D8312EC23503A031D8B
:100AE000602D831202308506EC23CA00473A031DAD
:100AF0005C2D8312EC23473A031D602D8312EC23F7
:100B0000413A031D602D8312B70A0319B80A1C303D
:100B10004023003803199C2D3C30F200F3011C30B7
:100B20004023F000F101552375083802031D9A2D6A
:100B300074083702031C602D8312861A2018A12D19
:100B4000602D0514EC233923EC23B900EC23BA0003
:100B5000EC23BB00EC23BC00EC23BD00EC23BE0067
:100B6000EC23BF003923EC23C0003923EC23C10060
:100B7000EC23C200EC23C300EC23C400EC23C5002B
:100B8000EC23C600EC23C700EC23C8003923EC2378
:100B9000C900EC23EC23303A0319D22D39082C3A42
:100BA000031DD72DC430B707031CB803602D831273
:100BB000EC2339233923A101A201A301A401A5013A
:100BC000A601EC23CB00CA012D3A83120319592E3A
:100BD0002508A6002408A5002308A4002208A300D5
:100BE0002108A2002130F1004B08D03E4923CC005F
:100BF000643083124C02031C1D2E9C30CC07A20AC9
:100C00000A302202031CF82DF630A207A30A0A308C
:100C10002302031CF82DF630A307A40A0A3024028D
:100C2000031CF82DF630A407A50A0A302502031C80
:100C30001B2EF630A507A60AF82D0A30F1004C0845
:100C400088274A07A1000A302102031C462EF630ED
:100C5000A107A20A0A302202031C462EF630A20780
:100C6000A30A0A302302031C462EF630A307A40A67
:100C70000A302402031C462EF630A407A50A0A30C7
:100C80002502031C462EF630A507A60A83124C083F
:100C9000CA000A304A02031C502EF630CA07492EF9
:100CA000EC23CB002C3A0319582E4B082E3AE52D95
:100CB0008312862420100230B700B801602D831201
:100CC000EC23543A031D602D8312EC23473A031D95
:100CD000602D8312EC233030D200D300CA0083127F
:100CE0005208D1005308D2004A08D300EC23CA00AE
:100CF0002E3A03197F2E4A082C3A031D6F2E8312B9
:100D0000EC234D3A8312031D802EEC233030D500A6
:100D1000D600CA0083125508D4005608D5004A08E8
:100D2000D600EC23CA002E3A03199A2E4A082C3A10
:100D3000031D8A2E1C30831240230038031D602DB2
:100D400054308C237008B5007108B60051308C23E4
:100D50007008B3007108B4004D304023F000F10179
:100D60007108803AF2003608803A7202031DBA2EEA
:100D700035087002031CCC2E3C308312F200F301C4
:100D80004C304023F000F10155237408B100750880
:100D9000B200AF01B001482F483083124023AD00AC
:100DA0004E304023F000F1017108803AF20036081D
:100DB000803A7202031DDE2E350870020318E62EFB
:100DC0004B3083124023B100B201102F4E308312FA
:100DD0004023F200F3014B304023F000F101552392
:100DE0007408F0007508F1003608F3003508F200C9
:100DF00073277408B1007508B2000A30F200F301DD
:100E000049304023F000F10155237408F0007508C3
:100E1000F1003608F3003508F20073277408AD07B7
:100E2000513083122D02031C172F5030AD00570A8A
:100E30000319580A031D202F3308D7003408D8009F
:100E400057083302AF005808031C580A3402B00098
:100E5000B01F322F33085702AF003408031C340A86
:100E60005802B0003008803AF00080307002B5308F
:100E700003192F02031C492F6830F0000130F100E4
:100E80002F087002AF003008031C300A7102B00056
:100E900083122D08F000F1017108803AF200300849
:100EA000803A7202031D562F2F0870020318652F17
:100EB0004A304023F000F10138087102031D622F0F
:100EC000370870028312031C6D2F38083202031D8D
:100ED0006B2F370831020318602D20143308D70018
:100EE0003408D800602DF601F11F7D2FF009F00ABB
:100EF0000319F103F1097617F61773088039F6061E
:100F0000F31FBF2FF209F20A0319F303F309BF2FEE
:100F1000F000F4010310FD307107031CAF2FF30143
:100F2000F0307105031D972F0430F300F10EF2012C
:100F30000310F30AF10D031C992FF10C71087002D4
:100F40000318F000F20DF30B9D2FF41FA92FF209E7
:100F5000F20A7208F41F0800F009F00A0800F10C08
:100F60000318B82FF10C031CF0010310F00C031C44
:100F700003107008F200F001F00DA52FF601F40146
:100F8000F50172087304031DC82FF001F10100344C
:100F90001F30F6040310F60AF20DF30D031CCB2FDD
:100FA000F30CF20C73087102031DD82F7208700243
:100FB000031CE02F7208F0027308031C730AF1028D
:100FC000F40DF50DF60BF61AD02FF61FEC2FF409E1
:100FD000F40A0319F503F5097408F2007508F30023
:100FE000761F0034F009F00A0319F103F109003407
:100FF000303430343034303430343034FF34FF3433
:02400E00663F0B
:104200008200A0008A00A400B000A20060009C0010
:104210009E0086008200980098006000A4008A003A
:1042200098008200B20040006000AE00920088005A
:104230008A00640040006500000032002F003E004C
:10424000000000000000000000000000000000006E
:10425000000000000000000000000000000000005E
:10426000000000000000000000000000000000004E
:10427000000000000000000000000000000000003E
:10428000000000000000000000000000000000002E
:0E4290001400190005005A001400030032004B
:00000001FF
